:10000000830100308A004728F60003088301D100ED
:100010008B1A0B1D40280B11FC3083120313810037
:10002000AD0A2D08043A031D3928AD01AE0AA11C02
:100030001D28AF0A031D1D28A117211D2328B00A62
:10004000031D23282214A11E3928C00A0319C10A3E
:1000500003304102E830031940020318A112C20A1A
:100060000319C30A013043022C300319420203185A
:100070002113211F4028051F3F280513402805177D
:100080000313831251088300F60E760E0900233005
:1000900084004F30542020308400233054208301CA
:1000A000F62D04068001840A0406031D512800343D
:1000B00083120313CF00D01B6628501B6E285008F4
:1000C0008A004F08CF0A0319D00A82008313501800
:1000D00083174F08CF0A8400000808003E345134CB
:1000E000493445343E34003442347F3440340034A3
:1000F0004234613451344934463421344134453436
:100100004B3431341834143412347F3410342734DF
:1001100045344534453439343C344A34493449341F
:1001200030340134713409340534033436344934FD
:1001300049344934363406344934493429341E3478
:1001400000340034003400340034083408340834F7
:100150000834083400340034C034C034003400346F
:1001600006340934093406343E34413441344134D0
:1001700022342034543454345434783440343834B1
:10018000043404347C34383444344434443438340F
:100190007C341034103410347C34273448344834E0
:1001A00048343F347C342034103408347C347C347C
:1001B000403440347C34C0343E34413441344134E2
:1001C0003E347C3454345434543424347C34143425
:1001D0001434143408347C345034203400347C34E7
:1001E0007C3454345434543428347F340834143434
:1001F00022344134223449344934493436340134C8
:1002000001347F3401340134383454345434543498
:1002100018347C340834103408347C347C3404348E
:10022000043404347C34043404347C34043404341E
:100230000C345034503450343C340034363436347A
:1002400000340034083400340834003408340034F6
:100250000834143422344134413422341434083400
:100260000034143414341434143414343F3440340B
:10027000403440343F347F3449344934493436348F
:100280007E341134113411347E347C341034103403
:1002900028344434283444345434543428344834CE
:1002A0003434143414347C346C3410347C341034CE
:1002B0006C341F342034403420341F347F344934AC
:1002C0004934493441347F340934193429344634AB
:1002D0007F3440344034403440347F340834083470
:0402E00008347F342B
:100682008A308301C400C40B442B0800023083016A
:10069200C600C60B4A2B080012308301C600C60BE7
:1006A200502B08009E308301C400C40B562B080057
:1006B2008301C80086128610402486140800830134
:1006C200CB00861686104024861408009630C1247A
:1006D2005A30C1246430C1249630C12C8301C70032
:1006E200460807394038592347087F398038592B43
:1006F200F0000030711870070310F00D0310F10CB8
:10070200F108031908007B2BFF30C1244B30C124B0
:10071200A030C1247830C124E130C124E630C12C9C
:1007220083012E08C5001930C5072E084502C400F2
:10073200C408031908006400962BF401F5010310A4
:10074200F30CF20C031CAC2B7008F40771080318AD
:10075200710AF5070310F00DF10D72087304031905
:100762000034A02B8301C60100306F23F830C4008F
:100772000130C500640000306023C4080319C503BA
:10078200C4034508803AF00080307002013003193A
:100792004402031C0800BB2BB430C124B430C12472
:1007A200B430C124B430C124B430C124B430C12423
:1007B200B430C124B430C124B430C124B430C12413
:1007C200B430C124B430C124B430C124B430C12CFB
:1007D20008308301C400C5016400061183160611A6
:1007E20000000000000006154723A0100619A014FF
:0E07F2004D230310C50CA01C002C8030C50741
:100800004723C40BED2B47234508080064008312DF
:100810000313861586140000861191238615213056
:100820005923C2305923073059231330592320301C
:10083000592309305923B323083059230C30592345
:10084000C60100306F2B08308301C400C50164006D
:10085000051283160512000000000000051647234C
:100860002011051A20154D230310C50C201D3A2C0C
:100870008030C5074723C40B272C472345080800B1
:100880008301CC0064000830CD00CE010612CC1FDD
:100890004B2C06144C2C061006160310CC0DCD085C
:1008A0000319CE03CD034E08803AF0008030700269
:1008B000013003194D02031C0800462C8301C400BB
:1008C0000830C500A0104418A014831203130611A9
:1008D0008316061100000000000000008312A01C17
:1008E000742C83160615762C831606114D23831659
:1008F000061547230310C40CC50B622C472B05308B
:100900008301C60000306F23D230C124D730C12408
:10091000D730C124AA30C1249B30C1243730C12430
:100920007830C1244B30C124DC30C1247830C1245C
:10093000E130C124E630C1249630C1245A30C12CA4
:100940008301C4000830C50020114418201583120B
:1009500003130512831605120000000000000000BA
:100960008312201DB62C83160516B82C831605128B
:100970004D238316051647230310C40CC50BA42C66
:10098000472B8301C400C900CA010530C700C80154
:100990004A08003ED00049086E3E0318D00A58208D
:1009A000C500C6016023C90A0319CA0AC70803198A
:1009B000C803C7034808803AF00080307002013055
:1009C000031947020318C82C0030602B0230830142
:1009D0009F0086018501BF3083168500C4308600E4
:1009E00080309F0020308B0083128C0183168C0195
:1009F00007308100FC30831281008B17A013A113F4
:100A0000A1102110221021112113A112A210C20144
:100A1000C3014208C0004308C100AD0108006400E2
:100A200083120313A401A30183160516061583126E
:100A30000512061183160512061153238316051697
:100A400006154D23A0110619A015831203132012B9
:100A5000051A20164123A0120619A01683120313AB
:100A60002013051A2017A01A372DA301A30A201B53
:100A70003B2DA401A40AA01D3F2D0230A307201E78
:100A8000472B0230A407472B8301C5004408BE0052
:100A9000BF01BF00BE014508BE04BF1F5F2D20146B
:100AA0003F08F1003E08F000F009F109013070073D
:100AB000BE000030031801307107BF00602D201008
:100AC0000530F200F3013F08F1003E08F0009E23DC
:100AD0007408B2007508B300A601A501A701320889
:100AE000BC003308BD003D08803AF0008030700241
:100AF0000A3003193C02031CA82DF6303C073D08C0
:100B000003183D0AFF3E8039031D8B2DA70AF630DE
:100B1000BC07031CBD032708F000F101F63E710875
:100B20000318710AFF3E8039031D992DA50AF6307E
:100B3000A7072508F000F101F63E71080318710AB5
:100B4000FF3E8039031D732DA60AF630A507732DCD
:100B50003C08BA003D08BB002708B800B9012508C9
:100B6000B600B7012608B400B501201CBA2D0B3021
:100B7000B400B501A608031D0800A508031DEC2D4F
:100B8000A708031DE12D3D083C04031DD42D0A30A8
:100B9000B800B901B6003908B7003608B400370804
:100BA000B500BA01BB010800201CD82D0B30D92D8F
:100BB0000A30B600B7010A30B400B501B801B90176
:100BC0000800201CE52D0B30E62D0A30B600B701D9
:100BD0000A30B400B5010800201CF22D0B30B4001F
:100BE000B50108000A30B400B50108006400E6242D
:100BF0000624803083169F008312B1012112A111B7
:100C00000030211A0130AC000030A1190130AC00D5
:100C10000030211A0130AC000030A2180130AC00C5
:100C20000030A11A0130AC000030211B0130AC00B3
:100C300047231F1F232E21162A2E1F1B2A2E831601
:100C40009F0A8312B10A4723640010303102031C4B
:100C50001D2EA115211AA42EA119962E0730F100E0
:100C60003108083E7923AC006400A501A701BC004F
:100C7000BD013D08803AF000803070020A3003194F
:100C80003C02031C612E6400F6303C073D0803184B
:100C90003D0AFF3E8039031D522EA70AF630BC07DD
:100CA000031CBD032708F000F101F63E710803188C
:100CB000710AFF3E8039031D392EA50AF630A707B9
:100CC000392E3C08B8003D08B9002708B600B70126
:100CD0002508B400B501A218742E0830310203189B
:100CE000732EA1162117A214A11ABA2E0530C60020
:100CF00000306F2385233C30C124C330C124350824
:100D000034040319882E0530F10034087923892E24
:100D10003230C1240530F10036087923C1243C303B
:100D2000C1240530F10038087923B42E0530C600FF
:100D300000306F2385236723BE30C1240530C124D2
:100D40001E30C124CD30B82EA218A92EA116A2148F
:100D50002117A11ABA2E0530C60000306F23852353
:100D60006723B930C1241E30C124CD30C1243230B4
:100D7000C124BB2E7F24C60100306F233230C12432
:100D80009130C1249630C1249B30C124A030C124AD
:100D90009630C1247830C1244B30C124A530C12401
:100DA000AA30C1247830C1244B30C1243230C12450
:100DB0003230C124C601C60A00306F23CD23023071
:100DC000C60000306F234630C1244B30C124503060
:100DD000C1245530C1245A30C124AF30C12403305E
:100DE000C60000306F235F30C1245030C12464300E
:100DF000C1246930C1244B30C124AF30C124043038
:100E0000C60000306F23CD238B130F258B172303D0
:100E10000319712F2308023A0319612F8B13CC3069
:100E20005E248B17A1181B2F8B1344305E248B1765
:100E3000A114AF01A113A118061D252FA11F252F55
:100E40008B13BE305E248B17A0179123A01F832F16
:100E50008B13E923A800E923AA008B17C4002808F4
:100E60004425A113A110A0130230C6002A306F231D
:100E70000530F10034087923C1240530F10036082B
:100E80007923C1240530F10038087923C124A6084C
:100E9000031D562FA508031D562FA708031D562F07
:100EA0003D083C04031D562F3230572F3C30C124DF
:100EB0000530F1003A087923C1244130C12446307D
:100EC000822F0230C6002A306F233230C1246E30A8
:100ED000C1247330C1247830C1247D30C1248230D4
:100EE000802F0230C6002A306F233230C124873071
:100EF000C1243C30C1248C30C1243C30C124323068
:100F0000C1243230C12424030319ED2F2408023AEE
:100F10000319DD2F8B13CC30A0248B172119972FA9
:100F20008B134430A0248B172115B00122102119F6
:100F3000051EA12F221CA12F8B13BE30A0248B17BE
:100F400021149123211CF92D8B132324A900232480
:100F5000AB008B17C4002908442522102111211051
:100F60000330C6002A306F230530F100340879239E
:100F7000C1240530F10036087923C1240530F10081
:100F800038087923C124A608031DD22FA508031D04
:100F9000D22FA708031DD22F3D083C04031DD22FDA
:100FA0003230D32F3C30C1240530F1003A08792388
:100FB000C1244130C1244630FE2F0330C6002A3000
:100FC0006F233230C1246E30C1247330C124783095
:100FD000C1247D30C1248230FC2F0330C6002A306A
:100FE0006F233230C1248730C1243C30C1248C307F
:100FF000C1243C30C1243230C1243230C124F92D07
:02400E003C3F35
:00000001FF
